:1000000005C1000030C100002EC100002CC100005D
:100010002AC1000028C1000026C1000024C1000040
:1000200022C1000020C100001EC100001CC1000050
:100030001AC1000018C1000016C1000014C1000060
:1000400012C100000C942F0D0EC100000CC1000065
:100050000AC1000008C1000006C100000C9452153E
:1000600002C100000C9494180C94D819FCC0000034
:10007000FAC00000F8C00000F6C00000F4C00000A4
:100080000C94020DF0C00000EEC00000ECC00000B7
:100090000C94D4180C94171AE6C000000C94F00EBF
:1000A000E2C00000E0C000000C94D50CDCC00000F1
:1000B000DAC00000D8C00000D6C000000C94A80C24
:1000C000D2C00000D0C00000CEC000000C941419B3
:1000D0000C94561AC8C000000C9454190C94951A2C
:1000E000C2C0000000002100240027002A002D00CB
:1000F0003000330001010000040107010A01000083
:100100002200250028002B002E00310034000201BF
:100110000000050108010B0100002000230026005B
:1001200029002C002F00320000010000030106010D
:10013000090105050505070508080808020202026D
:100140000A0A080804040404010101010101010173
:100150000303030303030303040707070C0C0C0C3E
:100160000C0C0C0C02020202060606060606060627
:100170000B0B0B0B0B0B0B0B0102102020080810B4
:100180002040102040800201020108040201010207
:1001900004081020408080402010080402018004E0
:1001A000020180402010080402010804020101023B
:1001B0000408102040800102040810204080000044
:1001C000090A02080B0C0D070603040100000000D9
:1001D000000000000000000000000000000000001F
:1001E0000000000000000000000011100F000000DF
:1001F00000000000000000000000000000000000FF
:10020000000000009701960D2112041C11241FBE4E
:10021000CFEFD1E2DEBFCDBF00E00CBF12E0A0E027
:10022000B2E0EEE9FCE300E00BBF02C007900D92E4
:10023000A03EB107D9F71BBE18E0A0EEB2E001C0A6
:100240001D92A73EB107E1F712E0CCE0D2E004C076
:100250002297FE010E94491EC430D107C9F70E94AF
:100260003A1D0C944D1ECCCEFB01DC014150504098
:1002700048F001900D920020C9F701C01D92415035
:100280005040E0F70895FC0181E090E001900616EF
:1002900009F4CF010020D1F701970895FB01519196
:1002A0005523A9F0BF01DC014D9145174111E1F73C
:1002B00059F4CD010190002049F04D9140154111B4
:1002C000C9F3FB014111EFCF81E090E00197089560
:1002D000482F803118F52091E0023091E102672B20
:1002E00081F481E090E002C0880F991F4A95E2F7FF
:1002F00080959095282339233093E1022093E002E2
:10030000089581E090E002C0880F991F4A95E2F7B6
:10031000282B392B3093E1022093E0020895893095
:1003200028F4E82FF0E0EE51FD4F60830895CF935D
:10033000DF93C2E1D4E0CE010E942F0A239684E02D
:10034000C23AD807C1F7DF91CF910895EF92FF929B
:100350000F931F93CF93DF93062F893008F078C057
:1003600090E00196682F660F660F660F019767345D
:1003700008F066E423E0880F991F2A95E1F7F82E2C
:10038000482FEE2451E0A02FB0E0C1E0D0E01EC025
:10039000842F82508434C0F4242F30E0F901EC50D3
:1003A000FD4F8081823080F4E52AF901EE0FFF1FB6
:1003B000ED5BFC4F11821082852F90E08A239B23F6
:1003C000892B11F0D183C083550F4F5F461700F37F
:1003D0001E2DE0FE05C0602F61708F2D0E94321827
:1003E00011FF06C0602F62708F2D8F5F0E94321840
:1003F00012FF06C0602F64708F2D8E5F0E9432182E
:1004000013FF06C0602F68708F2D8D5F0E94321819
:1004100014FF06C0602F60718F2D8C5F0E94321810
:1004200015FF06C0602F60728F2D8B5F0E943218FF
:1004300016FF06C0602F60748F2D8A5F0E943218ED
:10044000E7FE06C000788F2D895F602F0E9432186A
:10045000DF91CF911F910F91FF90EF9008950F932F
:100460001F93CF93DF93982F8B01863450F5C82FBD
:10047000D0E0FE01EC50FD4FE081E33091F0E4303C
:1004800001F592509033B8F49E0122503040C901DA
:10049000880F991F820F931F8E5E9B4F0E94CA0A7E
:1004A0000AC082508C3018F08A52833020F4892F91
:1004B000B8010E94A116CC0FDD1FCD5BDC4F198364
:1004C0000883DF91CF911F910F910895AF92BF9252
:1004D000DF92EF92FF920F931F93DF93CF930F92D0
:1004E000CDB7DEB7D82E7B01082F10E0F801EC5015
:1004F000FD4F8081863061F480910F04882341F0A4
:100500006630710529F010920F048FEF8093B802C6
:100510009D2D925099839033B0F4E4E0EE16F104EF
:1005200091F0C80102975C01AA0CBB1CA80EB91E71
:1005300082E194E0A80EB91EC5010E94B80A882382
:1005400011F0C501A6D74D2D46534031B8F4209186
:10055000E0023091E10292E0E916F10409F0D4C022
:1005600081E090E0042E02C0880F991F0A94E2F700
:10057000282B392B3093E1022093E002E981E43407
:1005800030F5ED2DE695E695E695980127703070EB
:10059000E114F10471F4F0E0E65CFC4F81E090E0DE
:1005A00002C0880F991F2A95E2F72081282B20830B
:1005B0000EC0F0E0E65CFC4F81E090E002C0880FE6
:1005C000991F2A95E2F78095208182238083F80184
:1005D000EE0FFF1FED5BFC4F11821082F2E0EF1671
:1005E000F104E1F083E0E816F1044CF4E114F104C5
:1005F00039F191E0E916F10409F07FC032C0E4E07E
:10060000EE16F10409F452C0F4E0EF16F104CCF157
:1006100086E0E816F10409F070C064C0403108F0CB
:1006200080C09981943440F48D2D60E00E947F1742
:100630008D2D60E00E9432180C501D4F82E05AC090
:10064000F981F43408F06DC08D2D60E00E947F17B1
:100650008D2D60E00E9432180C501D4FF801108261
:1006600060C0F981F43408F05CC08D2D60E00E9418
:1006700032188D2D61E00E947F170C501D4F81E0D4
:1006800039C0F981FC3028F08D2D8C52833008F070
:1006900048C08D2D61E00E947F178D2D60E070E0D5
:1006A0000E94A1160C501D4F83E024C0F981F03345
:1006B000C0F5F801EC50FD4F84E08083C80102973B
:1006C0007C01EE0CFF1CE80EF91E82E194E0E80EBE
:1006D000F91EC7014DD7882321F5C701B8010E9433
:1006E000E10B1FC09CEED90EE1E0ED15D0F00C50EF
:1006F0001D4F86E0F801808314C087EF95E060E02D
:1007000072E00E949D120DC081E090E0042E02C0B4
:10071000880F991F0A94E2F7809590952823392332
:1007200029CF0F90CF91DF911F910F91FF90EF9004
:10073000DF90BF90AF9008951F9380910F0488239E
:1007400029F010920F048FEF8093B80280E090E0C0
:10075000FC01EE51FD4F1082FC01E65CFC4F108263
:10076000FC01E551FD4F108201968930910581F71A
:1007700010E0812F8653803120F4812F62E070E0F9
:1007800003C0812F61E070E0A1DE1F5F163489F79E
:100790001092E1021092E0021F9108950F931F93AF
:1007A00007EF15E0C80161E172E042E023E00E943A
:1007B0009113C80160EE4FE252E00E94DD11C801C2
:1007C00060E946EA51E00E94DD11C80160EC48E6AC
:1007D00051E00E94DD11C80160ED4FE851E00E9438
:1007E000DD11C80164EF46E652E00E94DD11C80148
:1007F00060EF47EE57E00E940112C8016FEF4CE92D
:1008000053E00E94FB11C80140E051EE60E070E04F
:100810000E94041491DF1F910F9108951F9310E01F
:10082000812F8451823020F4812F66E070E04EDE0B
:100830001F5F1634A9F781E080930F048DE795E0E0
:100840000E942E0E1F9108951F93CF93DF93282FA0
:10085000162FC82FD0E0FE01E65CFC4F80811823E4
:10086000442331F4FE01E551FD4F8081811751F0A1
:1008700087EF95E0622F412F50E00E946F11C55124
:10088000DD4F1883DF91CF911F910895FF920F9351
:100890001F938091E2028823C1F1F0903A030F2D5B
:1008A000F2FE8CC282E00E946418892B09F486C291
:1008B00014E003FF06C083E00E946418892B09F04E
:1008C000186004FF06C084E00E946418892B09F0B8
:1008D000106105FF06C085E00E946418892B09F0AD
:1008E000106206FF06C086E00E946418892B09F09A
:1008F0001064F7FE06C087E00E946418892B09F097
:10090000106880E0612F40E09FDF8091E302882340
:1009100009F448C0F0903B030F2DF0FE51C288E06F
:100920000E946418892B09F44BC211E001FF06C034
:1009300089E00E946418892B09F0126002FF06C04A
:100940008AE00E946418892B09F0146003FF06C036
:100950008BE00E946418892B09F0186004FF06C020
:100960008CE00E946418892B09F0106105FF06C015
:100970008DE00E946418892B09F0106206FF06C002
:100980008EE00E946418892B09F01064F7FE06C0FF
:100990008FE00E946418892B09F0106881E0612FB4
:1009A00040E052DF8091E402882309F448C0F090CF
:1009B0003C030F2DF0FE06C280E10E946418892BD3
:1009C00009F400C211E001FF06C081E10E94641831
:1009D000892B09F0126002FF06C082E10E946418B0
:1009E000892B09F0146003FF06C083E10E9464189C
:1009F000892B09F0186004FF06C084E10E94641886
:100A0000892B09F0106105FF06C085E10E9464187A
:100A1000892B09F0106206FF06C086E10E94641867
:100A2000892B09F01064F7FE06C087E10E94641864
:100A3000892B09F0106882E0612F40E005DF80918A
:100A4000E502882309F448C0F0903D030F2DF0FE25
:100A5000BBC188E10E946418892B09F4B5C111E07B
:100A600001FF06C089E10E946418892B09F0126019
:100A700002FF06C08AE10E946418892B09F0146005
:100A800003FF06C08BE10E946418892B09F01860EF
:100A900004FF06C08CE10E946418892B09F01061E4
:100AA00005FF06C08DE10E946418892B09F01062D1
:100AB00006FF06C08EE10E946418892B09F01064BD
:100AC000F7FE06C08FE10E946418892B09F01068B8
:100AD00083E0612F40E0B8DE8091E602882309F4CC
:100AE00048C0F0903E030F2DF0FE70C180E20E94DE
:100AF0006418892B09F46AC111E001FF06C081E284
:100B00000E946418892B09F0126002FF06C082E27D
:100B10000E946418892B09F0146003FF06C083E269
:100B20000E946418892B09F0186004FF06C084E253
:100B30000E946418892B09F0106105FF06C085E248
:100B40000E946418892B09F0106206FF06C086E235
:100B50000E946418892B09F01064F7FE06C087E232
:100B60000E946418892B09F0106884E0612F40E02E
:100B70006BDE8091E702882309F448C0F0903F03C0
:100B80000F2DF0FE25C188E20E946418892B09F41C
:100B90001FC111E001FF06C089E20E946418892B81
:100BA00009F0126002FF06C08AE20E946418892BD5
:100BB00009F0146003FF06C08BE20E946418892BC1
:100BC00009F0186004FF06C08CE20E946418892BAB
:100BD00009F0106105FF06C08DE20E946418892BA0
:100BE00009F0106206FF06C08EE20E946418892B8D
:100BF00009F01064F7FE06C08FE20E946418892B8A
:100C000009F0106885E0612F40E01EDE8091E80267
:100C1000882309F448C0F09040030F2DF0FEDAC09D
:100C200080E30E946418892B09F4D4C011E001FF0D
:100C300006C081E30E946418892B09F0126002FF4C
:100C400006C082E30E946418892B09F0146003FF38
:100C500006C083E30E946418892B09F0186004FF22
:100C600006C084E30E946418892B09F0106105FF17
:100C700006C085E30E946418892B09F0106206FF04
:100C800006C086E30E946418892B09F01064F7FE01
:100C900006C087E30E946418892B09F0106886E07B
:100CA000612F40E0D1DD8091E902882309F448C03A
:100CB000F09041030F2DF0FE8FC088E30E9464186E
:100CC000892B09F489C011E001FF06C089E30E9465
:100CD0006418892B09F0126002FF06C08AE30E94A3
:100CE0006418892B09F0146003FF06C08BE30E948F
:100CF0006418892B09F0186004FF06C08CE30E9479
:100D00006418892B09F0106105FF06C08DE30E946D
:100D10006418892B09F0106206FF06C08EE30E945A
:100D20006418892B09F01064F7FE06C08FE30E9457
:100D30006418892B09F0106887E0612F40E084DD9A
:100D40008091EA02882309F44BC080914203082F66
:100D500080FF44C080E40E946418892B09F43EC0DF
:100D600011E001FF06C081E40E946418892B09F09C
:100D7000126002FF06C082E40E946418892B09F009
:100D8000146003FF06C083E40E946418892B09F0F5
:100D9000186004FF06C084E40E946418892B09F0DF
:100DA000106105FF06C085E40E946418892B09F0D4
:100DB000106288E0612F40E047DD12C010E079CD7D
:100DC00010E0B4CD10E0FFCD10E04ACE10E095CE9B
:100DD00010E0E0CE10E02BCF10E076CF10E0C1CFD6
:100DE0001F910F91FF900895EF92FF920F931F9321
:100DF000CF93DF93F82EEB01E42E8FEF6F3F780750
:100E000019F4C0E0D0E013C08DE795E06F2D54D603
:100E10008DE795E06C2FD1D68DE795E00FD78091C7
:100E2000100490911104009711F00E9401168DE7B3
:100E300095E06F2D4E2D10D70E2D10E08DE795E02B
:100E400045D60817190789F4F092EF03C093F00311
:100E5000C1EFD3E00C0F1D1F04C08DE795E03FD616
:100E60008993C017D107C9F711C08DE795E02ED639
:100E7000801791072CF487EF95E065E272E004C0DB
:100E800087EF95E06DE472E00E949D1282E0E80E2B
:100E900087EF95E067E74E2D2FEE33E00E94A1111A
:100EA000DF91CF911F910F91FF90EF900895AF9236
:100EB000BF92CF92DF92EF92FF920F931F93CF9347
:100EC000DF93E4DC04C087EF95E00E94E51287EF32
:100ED00095E00E944911892BB1F70E949A15609301
:100EE000CF037093D0038093D1039093D203A0904B
:100EF000D303B090D403C090D503D090D6032091F3
:100F0000B6023091B70279010027F7FC0095102F47
:100F10006A197B098C099D09E616F7060807190767
:100F200008F04AC0EA0CFB1C0C1D1D1DE092D30307
:100F3000F092D4030093D5031093D603C4EFD2E00C
:100F40001AEC1031C0F488818230A9F48091E0025B
:100F50009091E102012E02C0959587950A94E2F7DF
:100F600080FF09C0812F0E946D16AC0187EF95E0CC
:100F7000612F0E9455111F5F2196103111F780914A
:100F8000B80287FD19C010E00DC0F901EE0FFF1F78
:100F9000E20FF31FE952FC4F6181808170E04281D2
:100FA00023DF1F5F212F30E08091B802992787FD52
:100FB0009095821793074CF7DF91CF911F910F9176
:100FC000FF90EF90DF90CF90BF90AF900895BF92C9
:100FD000CF92DF92EF92FF920F931F93CF93DF9305
:100FE000162FEA018F3609F446C1803750F48B364C
:100FF00009F460C18D3609F4C1C1893609F025C2F2
:101000000CC2863769F0873720F4803709F01DC29B
:10101000DFC0883709F4C3C08A3709F016C210C18F
:10102000898185FF05C087EF95E064E772E050C0D5
:1010300068818871883041F1893018F4882341F043
:1010400004C2803109F43CC0883109F0FEC160C09F
:101050008DE795E031D502E00DC0FE01E00FF11DF6
:1010600061816795662767958081680F8DE795E0B8
:10107000A4D50E5F011788F38DE795E0DFD586E4F0
:1010800090E00E940116E1C19B818A81163071F4C3
:10109000979599279795980F4D81479544274795A0
:1010A0008C81480F862F692F70E008C0979599278B
:1010B0009795980F862F6FEF7FEF492F95DEC5C16B
:1010C0008091B80287303CF087EF95E060EA72E0EB
:1010D0000E949D12BAC18F5F8093B802992787FD45
:1010E0009095FC01EE0FFF1FE80FF91FE952FC4F2E
:1010F00060838B818795882787959A81890F818363
:101100008D818795882787959C81890F82839DC1D2
:101110005091B802151634F420E0C52FDD27C7FD25
:10112000D09511C08FEF8093B8028FC1FC01EE0FF4
:10113000FF1FE80FF91FE952FC4F6083662311F08F
:10114000422F24C02F5F822F90E0C817D90774F771
:1011500040E01CC04830C8F4C9010196D901AA0F6B
:10116000BB1FA20FB31FA952BC4FFC01EE0FFF1F04
:10117000E80FF91FE952FC4F80818C938081119612
:101180008C931197828112968C934F5F242F30E0BD
:10119000C217D307FCF651505093B80256C189814B
:1011A000682F70E07695762F66277795679588810A
:1011B000680F711D6115710521F070931104609322
:1011C000100480910F04882309F03FC127DB3DC143
:1011D000653008F43AC1F880C980EA80BB80DC80C1
:1011E0008F2D8250803308F030C10F2D10E0C801E0
:1011F0000297EC01CC0FDD1FC80FD91FCE5EDB4F6D
:10120000CE01B6D1882311F0CE0143D14E2D50E04E
:101210005695542F4427579547954C0D511D2D2D0C
:1012200030E03695322F2227379527952B0D311D2B
:10123000CE01B80116D28F2D64E070E047D905C108
:10124000623008F402C1898190E09695982F882732
:10125000979587952881820F911D9093B70280936F
:10126000B6020A970CF0F1C08AE090E09093B702C2
:101270008093B602EAC0623008F4E7C08981682F23
:1012800070E01230A1F08A8190E09695982F88271F
:1012900097958795682B792B133049F02B81922FE6
:1012A0009295990F990F907C80E0682B792B88811B
:1012B000D6D8CBC087EF95E060EF0E94D11187EFC1
:1012C00095E06CE60E94D1110EEF16C00434A0F434
:1012D00087EF95E060E00E94D11187EF95E061E033
:1012E0000E94D11187EF95E061E00E94D11187EF54
:1012F00095E061E00E94D111802F8453803150F439
:1013000087EF95E062E00E94D11187EF95E06AE0F7
:101310000E94D1110C3020F0802F8A52833050F47B
:1013200087EF95E063E00E94D11187EF95E068E0D8
:101330000E94D111003350F487EF95E064E00E94E1
:10134000D11187EF95E06EE00E94D111802F82517C
:10135000823050F487EF95E066E00E94D11187EF6C
:1013600095E061E00E94D11187EF95E06FE70E9460
:10137000D1110F5F043409F0A9CF63C0662309F4CB
:1013800064C0088187EF95E060EF0E94D11187EF7C
:1013900095E06EE60E94D11187EF95E0602F0E94E4
:1013A000D111063408F04DC0C02FD0E0FE01EC5042
:1013B000FD4F87EF95E06081F4D78E01000F111F7C
:1013C0000D5B1C4FF80160816F7787EF95E0E9D7DF
:1013D000F80160817181CB018078892B41F0660F23
:1013E000672F661F770B6F7787EF95E0DAD7CC0F03
:1013F000DD1FCD5BDC4F28813981C9018070907C75
:10140000892BF9F0330F220B330F322F221F622F5B
:101410006F7787EF95E0C5D714C087EF95E060EF51
:10142000C0D787EF95E06AE6BCD70AEC003110F030
:101430006FE701C0602F87EF95E0B3D70F5F0031F2
:10144000A9F787EF95E067EFACD7DF91CF911F91B8
:101450000F91FF90EF90DF90CF90BF900895FC0127
:101460008091A204803390F482838F5F8093A204E2
:10147000815090E0FC01EE0FFF1FE80FF91FED55C2
:10148000FB4F88EB9BE09283818308958FEF8283EB
:101490000895DC0112968C91129790E0FC01EE0FFA
:1014A000FF1FE80FF91FED55FB4F80818F7B808375
:1014B00012968C916CE00E94D71D90E0AC01440F15
:1014C000551F480F591F440F551F440F551F20E04B
:1014D00030E0C901840F951FFC01EE0FFF1FE80FDC
:1014E000F91FED55FB4F808186FD05C02F5F3F4FF3
:1014F0002C30310571F70895FC0122812033B8F5B5
:101500008081992787FD909548E850E0481B590B4A
:10151000440F551F440F551F6417750784F08181D0
:10152000992787FD909548E552E0481B590B440FD9
:10153000551F440F551F641775070CF4AB0142503B
:101540005040CA01AA2797FDA095BA2F880F991F6E
:10155000AA1FBB1F4FB7F89430E0F901EE0FFF1F31
:10156000E20FF31FED55FB4F928381834FBF089528
:10157000FC01828190E0FC01EE0FFF1FE80FF91FD4
:10158000ED55FB4F8081829586958695817009F097
:1015900081E00895AF92BF92CF92DF92EF92FF92D7
:1015A0000F931F93CF93DF93EC019B0182E0603296
:1015B00078070CF048C077FF03C020E030E005C09A
:1015C000653B710514F024EB30E000D00F92B901B7
:1015D000882777FD8095982F2881332727FD309520
:1015E000E8E8AE2EB12CA21AB30AAA0CBB1CAA0CB6
:1015F000BB1CCC24B7FCC094DC2CE981FF27E7FDA1
:10160000F09528E532E02E1B3F0B220F331F220FEF
:10161000331F442737FD4095542FEDB7FEB7218384
:1016200032834383548320E030E040E050E004EB19
:10163000E02EF12C012D112D0E94711D9B010F90A8
:101640000F900F900F90CE01B90156DFDF91CF912F
:101650001F910F91FF90EF90DF90CF90BF90AF90D0
:101660000895CF92DF92EF92FF921F93CF93DF9373
:10167000EC01162F7A0169018A81803308F093C04A
:10168000862F61E00E947F178A8190E0FC01EE0FB7
:10169000FF1FE80FF91FED55FB4F1F738081807C02
:1016A000812B808380E292E08E199F0964E070E0D4
:1016B0000E94E31D688380E699E08C199D0964E02F
:1016C00070E00E94E31D6983AA818A2F6CE00E946A
:1016D000D71D682F70E0AB01440F551F460F571FF1
:1016E000440F551F440F551F20E030E0C901840FFF
:1016F000951FFC01EE0FFF1FE80FF91FED55FB4F83
:10170000808186FD44C02F5F3F4F2C30310571F73B
:1017100053C01092800082E0809381001092850077
:1017200010928400B19A80916F00826080936F0064
:101730002EC06230710569F41092900082E08093AF
:101740009100109295001092940088BB80937100D4
:101750001EC06330710569F41092A00082E080938E
:10176000A1001092A5001092A40089BB8093720082
:101770000EC0672B61F41092200182E0809321015A
:1017800010922501109224018ABB809373008A2F46
:1017900090E0FC01EE0FFF1FE80FF91FED55FB4F26
:1017A0008081806480838A81DF91CF911F91FF9037
:1017B000EF90DF90CF9008956130710509F0B9CFB7
:1017C000A8CF40E252E020E639E04BCFEF92FF9203
:1017D0000F931F93CF93DF938B017A01EC01DC0110
:1017E000AD5CBA4F8C9187FF04C0FB01118210825F
:1017F00037C0AE01440F551F4C0F5D1F440F551FDE
:10180000440F551F2C91332727FD3095240F351F8A
:101810008091A20490E02817390714F58C9199273C
:1018200087FD9095840F951FFC01EE0FFF1FE80FB9
:10183000F91FED55FB4F808186FF12C08C919927CF
:1018400087FD9095840F951FFC01EE0FFF1FE80F99
:10185000F91FED55FB4F80818F7360E00E943218B5
:10186000DE01AD5CBA4F8C918F5F8C93AE01440F5B
:10187000551F4C0F5D1F440F551F440F551F2C91D2
:10188000332727FD3095240F351F8091A20490E067
:10189000281739070CF04DC08C918C300CF049C0E2
:1018A000F801208131818C91992787FD9095840FD3
:1018B000951FFC01EE0FFF1FE80FF91FED55FB4FC1
:1018C00081819281280F391FF701318320838C9108
:1018D000992787FD9095840F951FFC01EE0FFF1F40
:1018E000E80FF91FED55FB4F808186FF2AC08C91D0
:1018F000992787FD9095840F951FFC01EE0FFF1F20
:10190000E80FF91FED55FB4F80818F7361E00E9456
:10191000321817C080E49CE904C0F80180819181ED
:101920000496F70191838083CD5CDA4F8FEF888333
:1019300008C0F80180819181049680549C4950F33D
:10194000ECCFDF91CF911F910F91FF90EF90089511
:101950001F920F920FB60F920BB60F9211242F9376
:101960003F934F935F936F937F938F939F93AF9327
:10197000BF93EF93FF9380E090E064E271E048E270
:1019800051E024DFFF91EF91BF91AF919F918F9133
:101990007F916F915F914F913F912F910F900BBE6F
:1019A0000F900FBE0F901F9018951F920F920FB6B9
:1019B0000F920BB60F9211242F933F934F935F9387
:1019C0006F937F938F939F93AF93BF93EF93FF9307
:1019D00083E090E064EA70E048EA50E0F7DEFF91CF
:1019E000EF91BF91AF919F918F917F916F915F9197
:1019F0004F913F912F910F900BBE0F900FBE0F9004
:101A00001F9018951F920F920FB60F920BB60F9260
:101A100011242F933F934F935F936F937F938F93F3
:101A20009F93AF93BF93EF93FF9382E090E064E9BD
:101A300070E048E950E0CADEFF91EF91BF91AF91AD
:101A40009F918F917F916F915F914F913F912F91D6
:101A50000F900BBE0F900FBE0F901F9018951F9206
:101A60000F920FB60F920BB60F9211242F933F9344
:101A70004F935F936F937F938F939F93AF93BF9396
:101A8000EF93FF9381E090E064E870E048E850E075
:101A90009DDEFF91EF91BF91AF919F918F917F91CB
:101AA0006F915F914F913F912F910F900BBE0F90CF
:101AB0000FBE0F901F90189581E080937C05609376
:101AC000590510927A0510927B05089520915805CA
:101AD00030E080915705281B3109C90108954091D4
:101AE000570580915805481718F02FEF3FEF0AC0AF
:101AF000E42FF0E0E95CFA4F8081282F30E04F5F5F
:101B000040935705C9010895E09157058091580504
:101B1000E81718F0EFEFFFEF06C0F0E0E95CFA4FCE
:101B20008081E82FF0E0CF0108950895109280059C
:101B300010927F0588EE93E0A0E0B0E080938105ED
:101B400090938205A0938305B093840584EC92E082
:101B500090937E0580937D050895CF92DF92EF925A
:101B6000FF920F931F93CF93DF937C016B018A0148
:101B700080917C058823A1F0C0E0D0E00DC0D701A2
:101B8000ED91FC91D601AC0FBD1F0190F081E02DCD
:101B9000C7016C9119952196C017D10780F303C036
:101BA000CB01642F02D1C801DF91CF911F910F911A
:101BB000FF90EF90DF90CF900895DF93CF930F9237
:101BC000CDB7DEB7FC01698380917C058823C9F01D
:101BD00080917B05803238F081E090E093838283AE
:101BE00020E030E014C080917A05E82FF0E0E65A5A
:101BF000FA4F998190838F5F80937A0580937B055C
:101C000004C0CE01019661E0D0D021E030E0C901EE
:101C10000F90CF91DF9108950F93062F8091590572
:101C20006AE575E040917B0521E06AD010927A0563
:101C300010927B0510927C050F91089561E0ECCF26
:101C4000413208F040E2862F67E375E010D0109231
:101C5000570580935805089521E0F2CF109257055B
:101C60001092580510927A0510927B054EC2382FBB
:101C7000413210F040E042C0809189058823E1F7AD
:101C800091E09093890520938B058FEF8093F60563
:101C90001092B10541504093B2054F5F90938A0571
:101CA00080918A05330F832B80938A0580918C0560
:101CB000813041F410928C0580918A058093BB009D
:101CC00085EC01C085EE8093BC0080918905813050
:101CD000E1F38091B105841710F44091B10520E043
:101CE00030E00AC0FB01E20FF31FD901AF56BA4F33
:101CF0008C9180832F5F3F4F2417A0F3842F08958A
:101D00000F931F93582F122F413210F081E04AC0D9
:101D1000809189058823E1F782E08093890500930B
:101D20008B058FEF8093F6051092B1054093B205B5
:101D3000A1E9B5E0FB0102C081918D938E2F861B36
:101D40008417D0F310928A0580918A05550F852B50
:101D500080938A0580918C05813041F410928C0526
:101D600080918A058093BB0085EC01C085EE80934D
:101D7000BC00112321F0809189058230E1F380912C
:101D8000F6058F3F11F480E00DC08091F60580329A
:101D900011F482E007C08091F605803311F084E0F1
:101DA00001C083E01F910F910895482F613210F018
:101DB00081E0089580918905843011F082E00895D2
:101DC0006093D405A3EBB5E0842F9C01F90102C018
:101DD00081918D938E2F841B8617D0F380E0089518
:101DE0001F920F920FB60F920BB60F9211242F93E2
:101DF0003F934F935F936F937F938F939F93AF9393
:101E0000BF93EF93FF938091B90090E0887F90702B
:101E10008036910509F4F2C081369105CCF58832FF
:101E2000910509F47BC089329105B4F480319105A4
:101E300009F46FC0813191053CF4009709F447C162
:101E4000089709F04FC165C08831910509F466C053
:101E5000809709F047C182C08034910509F4A4C07D
:101E60008134910544F48033910509F482C0C89708
:101E700009F038C189C08035910509F489C08835D9
:101E8000910509F496C08834910509F02BC1AEC0C4
:101E90008839910509F413C189399105ECF4883723
:101EA000910509F4ABC0893791054CF4883691054A
:101EB00009F4A4C08037910509F014C19FC0883887
:101EC000910509F4FCC08039910509F49DC0803862
:101ED000910509F007C198C0803B910509F4C6C07F
:101EE000813B91054CF4803A910509F49FC0883AF2
:101EF000910509F0F7C0BAC0803C910509F4E3C030
:101F0000883C910509F4DFC0883B910509F0EAC0DF
:101F1000C2C080918A058093BB00CFC09091B1056B
:101F20008091B205981768F49091B105E92FF0E01F
:101F3000EF56FA4F80818093BB009F5F9093B1056D
:101F4000BCC080918B05882309F44BC085ED80933C
:101F5000BC008091BC0084FDFCCFC2C080E28093B5
:101F6000F60585ED8093BC008091BC0084FDFCCF1C
:101F7000B7C080E38093F60585ED8093BC00809127
:101F8000BC0084FDFCCFACC088E38093F6059BC009
:101F90008091B1059091BB00E82FF0E0EF56FA4F29
:101FA00090838F5F8093B1059091B1058091B205C8
:101FB00082C08091B1059091BB00E82FF0E0EF5610
:101FC000FA4F90838F5F8093B10580918B058823B2
:101FD00041F085ED8093BC008091BC0084FDFCCF76
:101FE0007FC081E080938C0584EA6EC085ED80938C
:101FF000BC008091BC0084FDFCCF72C083E0809364
:1020000089051092F50559C08091F505803208F0D8
:1020100056C08091F5059091BB00E82FF0E0EB529F
:10202000FA4F90838F5F8093F50547C08091F50547
:10203000803230F4E091F505F0E0EB52FA4F108277
:1020400085ED8093BC008091BC0084FDFCCF109294
:1020500089056091F505E0918F05F091900585ED7A
:1020600095E070E019951092F5052DC084E08093FD
:1020700089051092D3051092D405E0918D05F09159
:102080008E0519958091D405882329F481E08093E9
:10209000D4051092B3059091D305E92FF0E0ED54EB
:1020A000FA4F80818093BB009F5F9093D3059091FE
:1020B000D3058091D405981710F485EC01C085E80C
:1020C0008093BC000FC085EC8093BC0009C01092C7
:1020D000F60585ED8093BC008091BC0084FDFCCFAB
:1020E00010928905FF91EF91BF91AF919F918F91D0
:1020F0007F916F915F914F913F912F910F900BBE08
:102100000F900FBE0F901F9018951092890581E0D7
:1021100080938B0510928C0584E161E0A3D785E163
:1021200061E0A0D7E9EBF0E080818E7F8083808141
:102130008D7F808388E48093B80085E48093BC0021
:102140000895EF92FF920F931F937C018B01DC01A6
:10215000ED91FC91A081B1816F772D913C91CF01E0
:10216000F9011995D701ED91FC91A081B181000F82
:10217000012F001F110B0F772D913C91CF01602F84
:10218000F90119951F910F91FF90EF900895FC01AF
:102190000190F081E02DA081B1812D913C91CF0182
:1021A00060EFF90119950895FC010190F081E02D8F
:1021B000A081B1812D913C91CF0167EFF901199573
:1021C00008950F931F938C01DC01ED91FC91A08188
:1021D000B1812D913C91CF0169EFF9011995D80199
:1021E000ED91FC91A081B1812D913C91CF0162E0F4
:1021F000F9011995D801ED91FC91A081B1812D9142
:102200003C91CF0163E0F90119951F910F91089559
:102210001F93CF93DF93EC018A818823B1F1CE0124
:10222000B6DFE881F981A081B1812D913C91CF0188
:1022300069E7F9011995E881F981A081B1812B81C4
:102240003C814D915C91CF01F9016081FA011995B2
:10225000E881F981A081B1812B813C814D915C9114
:10226000CF01F9016181FA01199512E009C0EB81F2
:10227000FC81E10FF11D6081CE0170E062DF1F5F24
:102280008A811817A0F3CE018FDFDF91CF911F91C4
:102290000895FC01A081B181ED91FC91119704801A
:1022A000F581E02DCD0119950895EF92FF920F93DE
:1022B0001F938C017A01DC01ED91FC91A081B18129
:1022C0006F70606E2D913C91CF01F9011995C80195
:1022D000B70137DF1F910F91FF90EF900895EF92B4
:1022E000FF920F931F937C018A01DC01ED91FC9119
:1022F000A081B1816F7060692D913C91CF01F9018E
:102300001995D701ED91FC91A081B181602F6F7774
:102310002D913C91CF01F9011995D701ED91FC91D7
:10232000A081B181000F012F001F110B2D913C9155
:10233000CF01602FF90119951F910F91FF90EF9038
:102340000895DF92EF92FF920F931F93CF93DF9345
:10235000EC01162FD42E022FF32E19DFE881F9811C
:10236000A081B1812D913C91CF01612FF901199587
:10237000202F3F2DC9017C0110E007C0F7016191BA
:102380007F01CE0170E0DDDE1F5F1D15B8F3CE01C9
:102390000BDFDF91CF911F910F91FF90EF90DF90B6
:1023A0000895FC010190F081E02DA081B1812D9173
:1023B0003C91CF01F90119950895FC01603DA9F008
:1023C000613D28F4603959F0603CA1F40BC0603ED7
:1023D00019F0643F79F40CC054A743A7089556A799
:1023E00045A7089550AB47A7089552AB41AB089558
:1023F00054AB43AB0895FC016F3F11F456AB45ABB2
:102400000895FC0152AF41AF0895FC011582168278
:102410001782DC0180E018961C9218978F5F119646
:102420008032C9F710A612A611A605A8F6A9E02DBC
:10243000309709F019950895FC01128214821382D5
:10244000E4CF87EF95E0F8CF4F925F926F927F9243
:102450008F929F92AF92BF92CF92DF92EF92FF92B4
:102460000F93DF93CF930F920F92CDB7DEB72B016F
:102470007A013A8329838DE061E041D500E08981CA
:102480009A813C01882477FC8094982C5701CC24B5
:10249000B7FCC094DC2C0DC0C401B30159D38DE04E
:1024A00061E0E0D5C601B50153D38DE060E0DAD537
:1024B0000F5F802F90E08415950574F30F900F90B7
:1024C000CF91DF910F91FF90EF90DF90CF90BF9071
:1024D000AF909F908F907F906F905F904F900895F6
:1024E0000F931F938C018DE061E009D5C80162E074
:1024F00070E048E250E022ED30E0A6DF6AEF70E0E5
:1025000080E090E025D3C80163E070E048E250E04D
:1025100022ED30E099DF6DE770E080E090E018D3C5
:102520001F910F9108959A01FA0101900020E9F797
:102530003197E41BF50B4E2F04CFAB0161E7F3CFCE
:102540001F93CF93DF93EC018885813729F089377A
:1025500079F5CE015DDE35C08FA998AD892B89F163
:1025600089A59AA5019762E070E00E94E31D162FED
:10257000862F90E062D1AC01DC0121E030E011C097
:10258000FE01E20FF11D90859C932F5FFE01E20F8B
:10259000F11D8085879588278795890F8D932F5FFB
:1025A0003F5F311768F3EFA9F8ADCA01199509C06B
:1025B000E9ADFAAD309729F069A561502996AE01D1
:1025C0001995DF91CF911F910895CF93DF93EC017F
:1025D000A881B981ED91FC9111970680F781E02DDA
:1025E000CD011995AC0188A5882389F0473F510595
:1025F00021F418A6CE01A4DF91C089A59AA5FE01F9
:10260000E80FF91F408701969AA789A787C08D8197
:10261000882309F446C0403851050CF042C081506F
:102620008D83FE01E80FF11D4087882309F076C0F5
:102630008E81882309F472C0803D49F1813D28F4E0
:10264000803959F0803C59F51FC0803E19F0843F15
:1026500031F513C0EBA5FCA502C0EDA5FEA5309792
:10266000F1F0688570E07695762F66277795679507
:102670008985680F711D8F8111C0EBA9FCA9309766
:1026800071F06885898509C0EFA5F8A902C0E9A99C
:10269000FAA9309721F068858F8170E019951E8224
:1026A0003DC0403F510514F09A0106C09A01207FB9
:1026B0003070842F8F708F83203E3105F1F0213EE2
:1026C000310554F4203C3105D1F0203D3105B9F0FD
:1026D0002039310519F511C0243F310571F0253F2E
:1026E000310524F4203F3105C9F40DC0293F3105DF
:1026F00091F02F3F310591F40BC082E001C081E0E1
:102700008D832E830BC081E088A71AA619A606C068
:10271000CE017BDE03C087EF95E053DDDF91CF91E3
:102720000895AF92BF92CF92DF92EF92FF920F93F4
:102730001F93CF93DF938C01D62EC72EB42EA22EDB
:10274000862F972F61EB72E00E944E01EC018D2DD8
:102750009C2D6FE270E00E944301209779F07C018C
:102760000894E11CF11CE114F10441F09E012E5F7C
:10277000822F8E19D80112968C930FC0AD2DBC2DCF
:10278000FD0101900020E9F7ED19EF5FD8011296E5
:10279000EC932D2D3C2DC9017C01F801838194819E
:1027A000E9D0D80112968C9190E047D0FC01D80175
:1027B00014969C938E93139712968C911297E80F10
:1027C000F11D10821396ED91FC911497B08213962F
:1027D000ED91FC911497A18213968D919C91149781
:1027E00012964C9150E0425050400296B7010E9420
:1027F0003401DF91CF911F910F91FF90EF90DF9007
:10280000CF90BF90AF900895EF92FF920F931F93D8
:102810008C013BE5E32E38E0F32EC701C5D6F80165
:10282000F182E082C8015CDEC801CBDCC801F0DCCB
:102830001F910F91FF90EF9008950F931F93CF93E7
:10284000DF93BC018230910510F462E070E0E0910A
:10285000E508F091E608A0E0B0E040E050E024C0D8
:102860008081918186179707D0F08617970771F4BA
:1028700082819381109729F013969C938E931297DF
:102880002CC09093E6088093E50827C041155105B8
:1028900019F08417950718F4EF018D01AC01DF01E1
:1028A000828193819C01F9013097D1F64115510540
:1028B000F9F0CA01861B970B8430910580F48A8158
:1028C0009B810115110521F0F8019383828304C0D7
:1028D0009093E6088093E508FE01329645C0FE011C
:1028E000E80FF91F619371930297998388833CC025
:1028F0008091E3089091E408892B41F48091BB0218
:102900009091BC029093E4088093E3084091BD024B
:102910005091BE024115510541F44DB75EB780910B
:10292000B9029091BA02481B590B2091E3083091EB
:10293000E40824173507B0F4CA01821B930B8617ED
:10294000970780F0AB014E5F5F4F8417950750F0FB
:10295000420F531F5093E4084093E308F901619339
:10296000719302C0E0E0F0E0CF01DF91CF911F91C1
:102970000F910895CF93DF939C01009709F48FC0C6
:10298000EC0122971B821A826091E5087091E6089B
:102990006115710581F488819981820F931F2091BF
:1029A000E3083091E4082817390739F5D093E40893
:1029B000C093E30874C0DB0140E050E0AC17BD07F2
:1029C00008F1BB83AA83FE0121913191E20FF31F2D
:1029D000AE17BF0779F48D919C911197280F391F7D
:1029E0002E5F3F4F3983288312968D919C911397C8
:1029F0009B838A834115510571F4D093E608C093F7
:102A0000E5084DC012968D919C911397AD010097EA
:102A100011F0DC01D3CFDA011396DC93CE93129739
:102A2000FA0121913191E20FF31FCE17DF0769F40C
:102A300088819981280F391F2E5F3F4FFA0131831A
:102A400020838A819B8193838283E0E0F0E0DB0135
:102A500012968D919C911397009719F0BC01FD017E
:102A6000F6CFAB014E5F5F4FDB018D919C91840FE0
:102A7000951F2091E3083091E4082817390779F46D
:102A8000309729F41092E6081092E50802C01382EC
:102A90001282425050405093E4084093E308DF9183
:102AA000CF9108951F920F920FB60F9211242F937A
:102AB0003F938F939F93AF93BF93809136069091EE
:102AC0003706A0913806B091390630913A06019642
:102AD000A11DB11D232F2D5F2D3720F02D570196FD
:102AE000A11DB11D20933A068093360690933706B8
:102AF000A0933806B0933906809132069091330640
:102B0000A0913406B09135060196A11DB11D8093A8
:102B1000320690933306A0933406B0933506BF91E6
:102B2000AF919F918F913F912F910F900FBE0F907A
:102B30001F9018958FB7F89420913606309137067C
:102B400040913806509139068FBFB901CA010895E6
:102B50009B01AC017FB7F8948091320690913306C7
:102B6000A0913406B091350666B5A89B05C06F3FAD
:102B700019F00196A11DB11D7FBFBA2FA92F982F63
:102B80008827860F911DA11DB11D62E0880F991F36
:102B9000AA1FBB1F6A95D1F7BC012DC0FFB7F894DF
:102BA0008091320690913306A0913406B09135069B
:102BB000E6B5A89B05C0EF3F19F00196A11DB11D18
:102BC000FFBFBA2FA92F982F88278E0F911DA11D07
:102BD000B11DE2E0880F991FAA1FBB1FEA95D1F72C
:102BE000861B970B885E9340C8F2215030404040CE
:102BF000504068517C4F211531054105510571F652
:102C00000895019739F0880F991F880F991F02972F
:102C10000197F1F70895789484B5826084BD84B5F6
:102C2000816084BD85B5826085BD85B5816085BDC7
:102C3000EEE6F0E0808181608083E1E8F0E01082E0
:102C4000808182608083808181608083E0E8F0E021
:102C5000808181608083E1EBF0E08081846080830B
:102C6000E0EBF0E0808181608083E1E9F0E0808149
:102C700082608083808181608083E0E9F0E08081F0
:102C800081608083E1EAF0E08081826080838081DE
:102C900081608083E0EAF0E0808181608083E1E20E
:102CA000F1E0808182608083808181608083E0E2C6
:102CB000F1E0808181608083EAE7F0E080818460D8
:102CC0008083808182608083808181608083808135
:102CD000806880831092C1000895382F863308F0F1
:102CE000365320917B00832F86958695869590E0BC
:102CF0008170907043E0880F991F4A95E1F7277F14
:102D0000282B20937B0037708091BF028295880F1B
:102D1000880F807C832B80937C0080917A00806474
:102D200080937A0080917A0086FDFCCF2091780014
:102D300040917900942F80E030E0282B392BC90195
:102D400008951F93CF93DF93182FEB0161E0D7D045
:102D5000209709F4CAC0CF3FD10509F4C9C0E12FBB
:102D6000F0E0E254FE4F8491893009F466C08A3065
:102D7000B0F48430F1F1853040F4823059F1833081
:102D800070F5813009F0AEC020C0873009F443C02F
:102D9000883008F048C0863009F0A4C034C08D30B7
:102DA00009F478C08E3038F48B3009F45AC08C3076
:102DB00008F066C04CC0803109F480C0813109F44C
:102DC00087C08F3009F08EC06FC084B5806884BD25
:102DD000C7BD91C084B5806284BDC8BD8CC08091E0
:102DE0008000806880938000D0938900C093880021
:102DF00082C080918000806280938000D0938B009D
:102E0000C0938A0078C08091B00080688093B00041
:102E1000C093B30070C08091B00080628093B00016
:102E2000C093B40068C08091900080688093900047
:102E3000D0939900C09398005EC08091900080620A
:102E400080939000D0939B00C0939A0054C08091CF
:102E50009000886080939000D0939D00C0939C0068
:102E60004AC08091A00080688093A0008091A0005B
:102E70008F7B8093A000D093A900C093A8003BC093
:102E80008091A00080628093A000D093AB00C0939B
:102E9000AA0031C08091A00088608093A000D093E8
:102EA000AD00C093AC0027C0809120018068809362
:102EB0002001D0932901C09328011DC080912001D9
:102EC000806280932001D0932B01C0932A0113C00C
:102ED00080912001886080932001D0932D01C093C0
:102EE0002C0109C0C038D1051CF4812F60E002C05C
:102EF000812F61E0B7D0DF91CF911F910895CF93DB
:102F0000DF93482F50E0CA0188589E4FFC0134914E
:102F10004E5C5E4FFA018491882369F190E0880F3E
:102F2000991FFC01EC51FF4FA591B491FC01E250B7
:102F3000FF4FC591D491662351F42FB7F8948C912B
:102F4000932F909589238C93888189230BC06230BD
:102F500061F42FB7F8948C91932F909589238C93DB
:102F60008881832B88832FBF06C09FB7F8948C91EC
:102F7000832B8C939FBFDF91CF910895893009F403
:102F800049C08A30A0F4843051F1853040F4823059
:102F900079F1833000F5813009F063C026C08730B5
:102FA00079F1883098F5863009F05BC025C08D3006
:102FB00009F442C08E3028F48B30B1F18C30C0F56A
:102FC0002DC0803109F442C0813109F445C08F30F1
:102FD00009F047C037C0809180008F7703C080918F
:102FE00080008F7D80938000089584B58F7702C024
:102FF00084B58F7D84BD08958091B0008F7703C024
:103000008091B0008F7D8093B000089580919000F2
:103010008F7707C0809190008F7D03C080919000D2
:10302000877F8093900008958091A0008F7707C0DC
:103030008091A0008F7D03C08091A000877F809346
:10304000A0000895809120018F7703C08091200116
:103050008F7D80932001089580912001877F809348
:1030600020010895FF920F931F93F62E482F50E0F2
:10307000CA0182549E4FFC012491CA0188589E4F78
:10308000FC0114914E5C5E4FFA0104910023C1F0E3
:10309000222311F0822F72DFE02FF0E0EE0FFF1FEE
:1030A000E250FF4FA591B4919FB7F894FF2021F40F
:1030B0008C911095812302C08C91812B8C939FBFA2
:1030C0001F910F91FF9008950F931F93482F50E089
:1030D000CA0182549E4FFC012491CA0188589E4F18
:1030E000FC0104914E5C5E4FFA011491112319F416
:1030F00020E030E014C0222311F0822F3FDF812F27
:1031000090E0880F991F885E9E4FFC01A591B491B5
:103110008C9120E030E0802311F021E030E0C90103
:103120001F910F91089508951F920F920FB60F925D
:103130000BB60F9211242F933F934F938F939F932E
:10314000EF93FF938091C00082FD1DC04091C600A7
:1031500020917B0630917C062F5F3F4F2F7330709C
:1031600080917D0690917E062817390771F0E091D5
:103170007B06F0917C06E55CF94F408330937C063A
:1031800020937B0602C08091C600FF91EF919F9132
:103190008F914F913F912F910F900BBE0F900FBECB
:1031A0000F901F90189508951F920F920FB60F92CF
:1031B0000BB60F9211242F933F934F938F939F93AE
:1031C000EF93FF938091C80082FD1DC04091CE0017
:1031D00020910307309104072F5F3F4F2F7330700A
:1031E00080910507909106072817390771F0E09143
:1031F0000307F0910407ED53F94F40833093040720
:103200002093030702C08091CE00FF91EF919F9120
:103210008F914F913F912F910F900BBE0F900FBE4A
:103220000F901F90189508951F920F920FB60F924E
:103230000BB60F9211242F933F934F938F939F932D
:10324000EF93FF938091D00082FD1DC04091D60086
:1032500020918B0730918C072F5F3F4F2F73307079
:1032600080918D0790918E072817390771F0E091B2
:103270008B07F0918C07E55BF84F408330938C0708
:1032800020938B0702C08091D600FF91EF919F9110
:103290008F914F913F912F910F900BBE0F900FBECA
:1032A0000F901F90189508951F920F920FB60F92CE
:1032B0000BB60F9211242F933F934F938F939F93AD
:1032C000EF93FF938091300182FD1DC04091360144
:1032D00020911308309114082F5F3F4F2F733070E7
:1032E00080911508909116082817390771F0E09120
:1032F0001308F0911408ED52F84F408330931408EE
:103300002093130802C080913601FF91EF919F91A5
:103310008F914F913F912F910F900BBE0F900FBE49
:103320000F901F901895E0916708F0916808E05C95
:10333000FF4F8191919120813181821B930B8F737B
:103340009070892B09F0EFDEE0918908F0918A08EE
:10335000E05CFF4F8191919120813181821B930B21
:103360008F739070892B09F01EDFE091AB08F0910C
:10337000AC08E05CFF4F8191919120813181821BEB
:10338000930B8F739070892B09F04DDFE091CD087E
:10339000F091CE08E05CFF4F8191919120813181C5
:1033A000821B930B8F739070892B09F07CCF08954B
:1033B0001F920F920FB60F920BB60F9211242F93FC
:1033C0003F938F939F93EF93FF932091BF0630918C
:1033D000C0068091C1069091C2062817390731F4C2
:1033E0008091C1008F7D8093C10014C0E091C1061F
:1033F000F091C206E158F94F20818091C106909169
:10340000C20601968F7390709093C2068093C10696
:103410002093C600FF91EF919F918F913F912F9143
:103420000F900BBE0F900FBE0F901F9018951F921C
:103430000F920FB60F920BB60F9211242F933F935A
:103440008F939F93EF93FF93209147073091480705
:103450008091490790914A072817390731F48091E4
:10346000C9008F7D8093C90014C0E0914907F09195
:103470004A07E95FF84F20818091490790914A07F8
:1034800001968F73907090934A0780934907209319
:10349000CE00FF91EF919F918F913F912F910F90CF
:1034A0000BBE0F900FBE0F901F9018951F920F929A
:1034B0000FB60F920BB60F9211242F933F938F9359
:1034C0009F93EF93FF932091CF073091D007809186
:1034D000D1079091D2072817390731F48091D10094
:1034E0008F7D8093D10014C0E091D107F091D20775
:1034F000E157F84F20818091D1079091D207019632
:103500008F7390709093D2078093D1072093D60049
:10351000FF91EF919F918F913F912F910F900BBE53
:103520000F900FBE0F901F9018951F920F920FB61D
:103530000F920BB60F9211242F933F938F939F936B
:10354000EF93FF93209157083091580880915908C4
:1035500090915A082817390731F4809131018F7DF5
:103560008093310114C0E0915908F0915A08E95E46
:10357000F74F20818091590890915A0801968F73D6
:10358000907090935A088093590820933601FF91C8
:10359000EF919F918F913F912F910F900BBE0F90C4
:1035A0000FBE0F901F901895AF92BF92DF92EF92CF
:1035B000FF920F931F93CF93DF93EC017A018B015E
:1035C000DD24403081EE580780E0680780E078070E
:1035D00011F0DD24D39491E0A92EB12CEC89FD8962
:1035E000DD2069F0C50108A002C0880F991F0A9468
:1035F000E2F7808360E079E08DE390E005C010821F
:1036000060E874E88EE190E0A8019701EFD22150C4
:10361000304040405040569547953795279580E17A
:103620002030380720F0DD2011F0DD24D7CFE889E5
:10363000F9893083EA89FB89208319A2EE89FF8901
:10364000408121E030E0C9010C8C02C0880F991F35
:103650000A94E2F7482B4083EE89FF894081C90133
:103660000D8C02C0880F991F0A94E2F7482B408303
:10367000EE89FF894081C9010E8C02C0880F991F15
:103680000A94E2F7482B4083EE89FF8980810F8CF2
:1036900002C0220F331F0A94E2F7209528232083CB
:1036A000DF91CF911F910F91FF90EF90DF90BF902E
:1036B000AF900895DC011C96ED91FC911D97E05CA4
:1036C000FF4F2191319180819181281B390B2F73FC
:1036D0003070C9010895DC011C96ED91FC911D9795
:1036E000E05CFF4F20813181E054F040DF01AE5BB0
:1036F000BF4F8D919C9111972817390719F42FEF1F
:103700003FEF07C08D919C91E80FF91F8081282F12
:1037100030E0C9010895DC011C96ED91FC911D97E4
:10372000E05CFF4F20813181E054F040DF01AE5B6F
:10373000BF4F8D919C9111972817390719F42FEFDE
:103740003FEF10C08D919C911197E80FF91F2081D8
:103750008D919C91119701968F73907011969C9307
:103760008E9330E0C9010895DC0191968C91919778
:10377000882339F05496ED91FC915597808186FF0E
:10378000F9CF91961C920895CF93DF93EC01EE85CB
:10379000FF85E05CFF4F20813181E054F0402F5FD6
:1037A0003F4F2F733070DF01AE5BBF4F8D919C9107
:1037B000119728173907D1F3E05CFF4F8081918181
:1037C000E054F040E80FF91F6083EE85FF85E05C70
:1037D000FF4F31832083EE89FF89208181E090E0D3
:1037E0000F8C02C0880F991F0A94E2F7282B2083C0
:1037F00081E089A3EC89FD8980818064808381E0F8
:1038000090E0DF91CF9108951F9310925E0810927F
:103810005D0828EE33E040E050E020935F083093ED
:103820006008409361085093620864ED72E0709301
:103830005C0860935B088BE396E090936808809344
:1038400067088FE796E090936A088093690885EC93
:1038500090E090936C0880936B0884EC90E09093D8
:103860006E0880936D0880EC90E0909370088093D0
:103870006F0881EC90E0909372088093710882EC5D
:1038800090E0909374088093730886EC90E0909396
:1038900076088093750814E010937708B3E0B0932E
:1038A0007808A7E0A0937908F5E0F0937A08E1E0C2
:1038B000E0937B081092800810927F082093810883
:1038C00030938208409383085093840870937E0855
:1038D00060937D0883EC96E090938A088093890832
:1038E00087E097E090938C0880938B088DEC90E0B4
:1038F00090938E0880938D088CEC90E090939008C4
:1039000080938F0888EC90E09093920880939108C0
:1039100089EC90E090939408809393088AEC90E06F
:1039200090939608809395088EEC90E09093980879
:103930008093970810939908B0939A08A0939B08D6
:10394000F0939C08E0939D081092A2081092A108A1
:103950002093A3083093A4084093A5085093A60889
:103960007093A00860939F088BE497E09093AC0855
:103970008093AB088FE897E09093AE088093AD08F2
:1039800085ED90E09093B0088093AF0884ED90E0CF
:103990009093B2088093B10880ED90E09093B408C2
:1039A0008093B30881ED90E09093B6088093B508BA
:1039B00082ED90E09093B8088093B70886ED90E090
:1039C0009093BA088093B9081093BB08B093BC08D1
:1039D000A093BD08F093BE08E093BF081092C408FE
:1039E0001092C3082093C5083093C6084093C708B7
:1039F0005093C8087093C2086093C10883ED97E0A4
:103A00009093CE088093CD0887E198E09093D008FA
:103A10008093CF0885E391E09093D2088093D108FA
:103A200084E391E09093D4088093D30880E391E0FD
:103A30009093D6088093D50881E391E09093D808BD
:103A40008093D70882E391E09093DA088093D908B5
:103A500086E391E09093DC088093DB081093DD0807
:103A6000B093DE08A093DF08F093E008E093E1084C
:103A70001F910895CF93DF93CED80E94CE03C3E960
:103A8000D9E10E9457072097E1F34DDCFACFCF929E
:103A9000DF92EF92FF920F931F93CF93DF937C01FE
:103AA0006B018A01C0E0D0E00FC0D6016D916D01BD
:103AB000D701ED91FC910190F081E02DC70119959E
:103AC000C80FD91F015010400115110571F7CE0123
:103AD000DF91CF911F910F91FF90EF90DF90CF90EA
:103AE00008952F923F924F925F926F927F928F92A2
:103AF0009F92AF92BF92CF92DF92EF92FF920F937D
:103B00001F93DF93CF93CDB7DEB73B014C01190173
:103B10002A016E897F89888D998D6A197B098C09A4
:103B20009D09621A730A840A950AA401930120D0A0
:103B3000E218F30804091509A801970179D02A0DA4
:103B40003B1D4C1D5D1DB901CA01CF91DF911F9135
:103B50000F91FF90EF90DF90CF90BF90AF909F902C
:103B60008F907F906F905F904F903F902F9008952F
:103B7000629FD001739FF001829FE00DF11D649F51
:103B8000E00DF11D929FF00D839FF00D749FF00DDD
:103B9000659FF00D9927729FB00DE11DF91F639F7E
:103BA000B00DE11DF91FBD01CF0111240895991B2E
:103BB00079E004C0991F961708F0961B881F7A9524
:103BC000C9F78095089597FB092E07260AD077FD3F
:103BD00004D049D006D000201AF4709561957F4F2B
:103BE0000895F6F7909581959F4F0895A1E21A2EBA
:103BF000AA1BBB1BFD010DC0AA1FBB1FEE1FFF1F91
:103C0000A217B307E407F50720F0A21BB30BE40BE0
:103C1000F50B661F771F881F991F1A9469F7609527
:103C20007095809590959B01AC01BD01CF010895E1
:103C300097FB092E05260ED057FD04D0D7DF0AD0FA
:103C4000001C38F450954095309521953F4F4F4FCB
:103C50005F4F0895F6F790958095709561957F4F29
:103C60008F4F9F4F0895AA1BBB1B51E107C0AA1F8E
:103C7000BB1FA617B70710F0A61BB70B881F991F0D
:103C80005A95A9F780959095BC01CD010895EE0F46
:0E3C9000FF1F0590F491E02D1994F894FFCFDA
:103C9E00556E6B6E6F776E2070696E206D6F6465FA
:103CAE00005374616E646172644669726D61746111
:103CBE002E696E6F00493243205265616420457251
:103CCE00726F723A20546F6F206D616E7920627937
:103CDE007465732072656365697665640049324365
:103CEE002052656164204572726F723A20546F6F74
:103CFE0020666577206279746573207265636569E5
:103D0E007665640031302D62697420616464726579
:103D1E007373696E67206D6F6465206973206E6FB3
:103D2E00742079657420737570706F727465640099
:103D3E00746F6F206D616E79207175657269657330
:103D4E00002E637070001300FF8000E70800000172
:103D5E0000000000DD0DAD0D660D6F0D840D950D8F
:103D6E0000000000C41B471D5A1B8B1B6B1BB41B92
:00000001FF
